:04000000B2017229AE
:100008000800B216B21EB212B2190E28B215472055
:10001800031835280830A3005B20A20DA30B102875
:10002800B21E402065206120B21A35203A202208ED
:1000380003106D29B216B21EB21232192828FE39E1
:10004800B300321503106D29321A3028A600321673
:1000580047200318352826084E2003183528B21ED5
:100068006D294020652032113212B2113608840001
:10007800340884178004462836088400340980052B
:100088008417800508003A20652040206120330845
:10009800B2190138A2000830A300A20D03183A20B3
:1000A800031C402065206120A30B51283A206520BD
:1000B8003608840034080005FF3E370884003509F7
:1000C80043283708840035083D280408A600360868
:1000D80084008030B3050830A70003100318B30A62
:1000E8008320A60CA70B72280000AB1A330C8320C0
:1000F8007021031483202F08A3002E0825298413B8
:10010800AB1F9228000834042B1F34068000841784
:1001180000083404031C340680009D2800083404B9
:10012800031C34062B1B3406800084173409800511
:100138009D282B081F39003EA1002A08083E0318F5
:10014800A10A00003229B31329080319B317043090
:10015800A800250EB4202508B420240EB4202408B5
:100168000F39F63E0318073E0A3EBA28A000A80336
:100178000319B31329080319C4282802031808000F
:100188002008031DB313B31B0800303E682908304C
:10019800A600A70037088400350833191821331D35
:1001A8001A213608840034081D21A001A10126085F
:1001B80003196D29B3180F21360884000008340587
:1001C800FF3EA00DA10DB31C0F21A60BDE282708AA
:1001D8003318462920086D290830A60037088400FE
:1001E800350833191821331D1A21360884003409BB
:1001F8002121260803196D29331846213608840061
:10020800A10CA00C00083404031C340680000F2144
:10021800A60B02296D2937088400350880060000DE
:10022800152916298006080080042029FF3A800530
:100238002129841780046D29FF3A841780056D29C8
:10024800A301A200FF30A207031CA307031C6D290A
:100258000330A100E43032212629A101F63EA00096
:10026800A109031C3D29FE300000A0070318382906
:10027800A0076400A10F372900002018432920187F
:1002880045290800A201A3014D29A10CA00CA20D2B
:10029800A30DFF3E031849292308A1002208A00046
:1002A8006D29A20001305829A80023082102031D46
:1002B8005F29220820020430031801300319023094
:1002C8002805031DFF306D29840031088A00300895
:1002D8008200831303138312640008008316073017
:1002E8009F0007148710071187128312D601D301C4
:1002F800B801B9010130A300F4308A012521073083
:10030800B6004030B4002030AA00AB01AE01AF0106
:1003180053308A016A2074308A016A2061308A0168
:100328006A2072308A016A2074308A016A200A3091
:100338008A016A200D308A016A208A110A12BF2CAC
:100348008716FF30D1000A30CF008A110A12D9234C
:10035800871232308A0124214030CE009530D000F7
:100368004E08D1000730B6000430B4000730B7009B
:100378000230B5000130B3005108A000A1018A0184
:10038800F020D1010430CF008A110A12D923500875
:10039800D1000730B6000430B4000730B70002308F
:1003A800B5000130B3005108A000A1018A01F02076
:1003B8000130CD008A110A124E22871632308A0186
:1003C8002421871264005708003C8A110A12031975
:1003D800242A8716FF30D1000730B6000430B40055
:1003E8000730B7000230B5000130B3005108A00053
:1003F800A1018A01F0208A110A1243248712413090
:10040800D1000730B6000430B4000730B70002301E
:10041800B5000130B3005108A000A1018A01F02005
:10042800D1010430CF008A110A12D923FF30D1003C
:100438008A110A1224248A110A1243248A01E629FD
:10044800FF30D1000730B6004030B4002030AA0099
:10045800AB01AE01AF0149308A016A204E308A01F2
:100468006A2049308A016A2054308A016A20203083
:100478008A016A204F308A016A204B308A016A203B
:1004880021308A016A200A308A016A200D308A01E7
:100498006A200800640057084D028A110A120319DD
:1004A800632A0730B6000130B4000730B7000230C5
:1004B800B500B3018A01CB20D7008A014E2A080073
:1004C8008716FF30CC008A110A1233248A110A12C7
:1004D800432487125830C8003B08C9003A08CA00AC
:1004E8003D08CB003C08CC008A110A12F723FF30E4
:1004F800CC008A110A1233248A110A124324CD012E
:100508008A014E22FE30CC008A110A123324400898
:10051800B8004108B9003808A0003908A10043080C
:10052800A30042088A0155218A110A12031DC62A0E
:100538000730B6001030B4000730B7000830B500F7
:10054800A0308A01202039088A01202038088A0131
:1005580020208A010520D1000730B6000430B400FD
:100568000730B7000230B5000130B3005108A000D1
:10057800A1018A01F020B80A0319B90A8A110A12DE
:10058800031D8F2AFF30D1000230CF008A110A12D2
:10059800D9238A110A1243240F305705D9008A112A
:1005A8000A12432464005708003C8A110A12031DEA
:1005B800EB2A0730B6000130B4000730B70002302C
:1005C800B500B3018A01CB20D7008A01D62A8A1147
:1005D8000A12A12308008716FF30CC008A110A12DC
:1005E80033248A110A12432487125130C8003B0869
:1005F800C9003A08CA003D08CB003C08CC008A1163
:100608000A12F723FF30CC008A110A1233248A1108
:100618000A124324CD018A014E22FE30CD008A0100
:100628004E224008BE004108BF003E08A0003F0817
:10063800A1004308A30042088A0155218A110A1221
:10064800031D4D2B0730B6000130B4000730B7004A
:100658000230B500B3018A01CB20D1000730B600C3
:100668001030B4000730B7000830B500A0308A0158
:1006780020203F088A0120203E088A0120205108B6
:100688008A011E20BE0A0319BF0A8A110A12031D15
:10069800192B8A110A1243248A110A1243248A1137
:1006A8000A12A12308005030CE00FF30D0008A1172
:1006B8000A12742308006030CE008A110A127423CB
:1006C80008006130CE008A110A1274230800013034
:1006D800D3006630CE008A110A127423D3010800B1
:1006E8008716FF30CC008A110A1233248A110A12A5
:1006F800432487124E08C8003B08C9003A08CA00BC
:100708003D08CB003C08CC008A110A12F723FF30C1
:10071800D1000230CF008A110A12D9238A110A1295
:10072800432464005308013C8A110A12031D9D2BBF
:100738000800CD018A014E2208008716FF30D1003B
:100748000730B6000430B4000730B7000230B500F7
:100758000130B3005108A000A1018A01F0208A11DC
:100768000A12432487124D30CC008A110A1233240E
:10077800D1010430CF008A110A12D923FF30CC00EE
:100788008A110A1233240730B6000130B40007304A
:10079800B7000230B500B30110308A01CC20C40084
:1007A8002108C5004408D60008000130D9006400BB
:1007B80059084F028A110A12031CF62B0730B6009B
:1007C8000430B4000730B7000230B5000130B30080
:1007D8005108A000A1018A01F020D90A8A110A1241
:1007E800031DDB2B08000730B6000430B4000730C7
:1007F800B7000230B5000130B3004808A000A101DD
:100808008A01F0200730B6000430B4000730B70082
:100818000230B5000130B3004908A000A1018A01E7
:10082800F0200730B6000430B4000730B7000230BB
:10083800B5000130B3004A08A000A1018A01F020E8
:100848000730B6000430B4000730B7000230B500F6
:100858000130B3004B08A000A1018A01F020073045
:10086800B6000430B4000730B7000230B5000130DC
:10087800B3004C08A000A1018A01F020080007304D
:10088800B6000130B4000730B7000230B500B3013C
:100898008A01CB20D70008000730B6004030B400EA
:1008A8002030AA00AB01AE01AF0144308A016A20B2
:1008B80061308A016A2074308A016A2061308A01B5
:1008C8006A2020308A016A2066308A016A207230E4
:1008D8008A016A206F308A016A206D308A016A2095
:1008E80020308A016A204D308A016A204D308A0101
:1008F8006A2043308A016A200A308A016A200D3052
:100908008A016A204008BE004108BF003E08A000D6
:100918003F08A1004308A30042088A0155218A1113
:100928000A12031DBE2C0730B6001030B400073081
:10093800B7000830B500A0308A0120203F088A019E
:1009480020203E088A0120208A010520D100073096
:10095800B6004030B4002030AA00AB01AE01AF01B0
:1009680051088A016A20BE0A0319BF0A8A110A12AD
:10097800031D8A2C08008A01A421BA01BB01BC010D
:100988000230BD008A015723C001C101FF30C200F7
:100998000130C3004130D1004008BE004108BF000B
:1009A8003E08A0003F08A1004308A30042088A01AE
:1009B80055218A110A12031DFC2C0730B60010308D
:1009C800B4000730B7000830B500A0308A012020F5
:1009D8003F088A0120203E088A01202051088A0108
:1009E8001E20BE0A0319BF0A8A110A12031DD42C3D
:1009F8000130BA00BB01BC01BD018A016422073085
:100A0800B6004030B4002030AA00AB01AE01AF01FF
:100A180044308A016A2061308A016A2074308A0170
:100A28006A2061308A016A2020308A016A205730A2
:100A38008A016A2072308A016A2069308A016A2034
:100A480074308A016A2074308A016A2065308A010C
:100A58006A206E308A016A2020308A016A20743048
:100A68008A016A206F308A016A2020308A016A2050
:100A78004D308A016A204D308A016A2043308A014C
:100A88006A200A308A016A200D308A016A208A01A8
:100A9800EF228A0150240730B6004030B4002030DD
:100AA800AA00AB01AE01AF010A308A016A200D30FD
:100AB8008A016A2045308A016A2072308A016A20D8
:100AC80061308A016A2073308A016A2069308A019C
:100AD8006A206E308A016A2067308A016A202E30C7
:100AE8008A016A202E308A016A202E308A016A2003
:100AF8000A308A016A200D308A016A208A015F2340
:100B08000130BA00BB01FF30BC000130BD008A01D2
:100B180065238A016B23BC01BD018A01EF220730DE
:100B2800B6004030B4002030AA00AB01AE01AF01DE
:100B380044308A016A2061308A016A2074308A014F
:100B48006A2061308A016A2020308A016A20663072
:100B58008A016A2072308A016A206F308A016A200D
:100B68006D308A016A2020308A016A204D308A015E
:100B78006A204D308A016A2043308A016A20203079
:100B88008A016A2061308A016A2066308A016A20F7
:100B980074308A016A2065308A016A2072308A01BD
:100BA8006A2020308A016A2065308A016A20723002
:100BB8008A016A2061308A016A2073308A016A20BA
:100BC80065308A016A200A308A016A200D308A015C
:100BD8006A204008BE004108BF003E08A0003F0848
:100BE800A1004308A30042088A0155218A110A126C
:100BF800031D2C2E0730B6001030B4000730B700A4
:100C08000830B500A0308A0120203F088A01202042
:100C18003E088A0120208A010520D1000730B6004D
:100C28004030B4002030AA00AB01AE01AF01023061
:100C3800A9005108A400A5016930B000B1018A01DA
:100C4800A720BE0A0319BF0A8A110A12031DF12D33
:100C58000730B6004030B4002030AA00AB01AE0126
:100C6800AF010A308A016A200D308A016A204130BA
:100C78008A016A206C308A016A206C308A016A20F5
:100C880020308A016A2044308A016A206F308A0144
:100C98006A206E308A016A2065308A016A20213014
:100CA8008A016A200A308A016A200D308A016A2086
:060CB80063008A015C2EBE
:02400E003D3D36
:00000001FF
